:020000040000FA
:1000000018290408A2008316051083120930A300E2
:1000100003101120A20CA30B0928031411200314B0
:10002000132903181628000005141828051018288D
:100030000030A1006230B728B31329080319B317A1
:100040000530A8002730A300103032200330A30071
:10005000E8303220A30164303220A3010A3032207C
:1000600024083928A2002508A1002408A000F220B5
:100070002008A000A8030319B31329080319432873
:100080002802031808002008031DB313B31B08003F
:10009000303E0E29A3003608840034097A208413E8
:1000A000A30803191329F030A50022088038A40002
:1000B000F030A5030319A5000319A303031913299D
:1000C0002008A6002108A7001630B6202608A000A8
:1000D0002708A1008420030120183408A21F340837
:1000E000A20803190301A40F772880065528782851
:1000F0000000582884178005132983178001840A7B
:10010000FF3E031D7E281329210820040319A00A9D
:100110008030201AA1062019A106A018A106210DE1
:10012000A00DA10D132903178D0083168C130C1439
:1001300083120C08132903178C0083168C130C15DB
:1001400055308D00AA308D008C148C18A5280C1108
:100150001329A301A200FF30A207031CA307031C5D
:1001600013290330A100E330B720AB28A101F43EEE
:10017000A000A109FE30031CC028A0070318BD2859
:10018000A0076400A10FBD2800002018C728201870
:10019000C9280800013EA7000A30A200A301F220EE
:1001A000A70BCF2824080800A2000330E228A200F1
:1001B0000130E228A2000630E228A2000430E22842
:1001C000A2000530A80023082102031DE928220807
:1001D0002002043003180130031902302805031DE2
:1001E000FF301329A501A4011030A600210DA40D94
:1001F000A50D2208A4022308031C230FA50203183F
:1002000008292208A40723080318230FA5070310B1
:10021000A00DA10DA60BF628200813298400310893
:100220008A003008820083130313831264000800DD
:1002300083167E308F0007309C009D01831297014A
:100240009001831690011F3085008601831283166A
:100250009F0183129F0183169B01643083128A01E0
:10026000A92064308A01A9202030840060308A01EE
:100270007E20A030840050308A017E20103084001F
:1002800060308A017D209030840060308A017D20BA
:1002900064308A01A9208516831685120D308312D9
:1002A0008A0102200A308A010220851383168513F1
:1002B0008312051383160513831286138316861380
:1002C00083120130A300F4308A01AA2001308A0190
:1002D0009320C200C3014208D6004308D700C20AD7
:1002E0000319C30A031701308D00031342088A0162
:1002F0009B20851783168513831205178316051314
:10030000831286010530A300DC308A01AA20851300
:100310008316851383120513831605138312093080
:10032000D800D9015808A0005908A100A301003045
:100330008A01DD208A11031DD2298A11FF22851727
:100340008316851306308312B6008030B400323035
:10035000A2000A308A014A208A11272314308A0118
:10036000A920851383168513831205178316051399
:1003700006308312B6008030B4003230A2000A305A
:100380008A014A208A11272314308A01A9200513E3
:100390008316051301308312D802031CD9028A1177
:1003A000031892293730D800D9015808A0005908FD
:1003B000A100A3017F308A01D7208A11031D042ADE
:1003C00085178316851306308312B6008030B4007B
:1003D0005808A20004308A014A2005178316051325
:1003E00083128830860001308A01A9208513831684
:1003F000851383120513831605138312D80A031974
:10040000D90A8A11031DD52942308A0102204F30B2
:100410008A0102204D308A01022042308A010220E6
:1004200020308A01022047308A01022041308A01AF
:1004300002204D308A01022045308A0102202030FE
:100440008A01022056308A01022031308A010220BE
:100450002E308A01022030308A01022020308A01A9
:10046000022020308A01022020308A010220283018
:100470008A01022020308A010220A9015608A40026
:100480005708A5000130B000B1018A011C202030BE
:100490008A01022029308A01022020308A010220AC
:1004A0000D308A0102200A308A0102200D308A01B3
:1004B00002200A308A0102204D308A010220413098
:1004C0008A01022044308A01022045308A0102203C
:1004D00020308A01022042308A01022059308A01EC
:1004E000022020308A01022052308A010220553039
:1004F0008A01022049308A01022020308A0102202C
:1005000043308A01022041308A01022042308A01B0
:10051000022052308A01022041308A0102204C30F0
:100520008A01022020308A01022032308A01022012
:1005300030308A01022031308A01022030308A01B5
:100540000220D601D701C601C701CA01CB01C401EF
:10055000C501D801D9014E08A0004F08A1008A01A9
:1005600084202008CE002108CF0020308A010220FC
:1005700053308A01022054308A01022041308A011E
:10058000022052308A01022054308A0102202E308B
:100590008A0102202E308A0102202E308A01022098
:1005A0000D308A0102200A308A0102208517831645
:1005B00085138312BB30860005308A01A92085137C
:1005C000831685138312FF308600051783160513E3
:1005D0008312C130860005308A01A92005138316D5
:1005E00005138312FF30860064008A11851CFD2AE2
:1005F0003230D000D1018A11552D8A01A32A590821
:100600008A11031D1C2B5808093C8A11031C1C2B42
:100610008A110E23CC00CD018A111C2B03308A00D5
:1006200058088207773444346B346E345C343E347B
:100630003F3464347F347C34FF30CC060030CD0648
:1006400064008A11851C262B8A112F230800FF3095
:10065000860001308A01A9204C088600080058084D
:10066000D6005908D7000830D800D90164008A1193
:10067000851C672B85178316851383120517831630
:100680000513831259088A11031D5F2B5808093C72
:100690008A11031C5F2B8A115123CC00CD018A11D2
:1006A0005F2B03308A0058088207773444346B3458
:1006B0006E345C343E343F3464347F347C34FF30F9
:1006C000CC060030CD068A0127238A01362B560836
:1006D000D8005708D90008008A11552D20308A010A
:1006E000022057308A01022041308A010220523014
:1006F0008A0102204E308A01022049308A010220FC
:100700004E308A01022047308A0102202E308A01B1
:1007100002202E308A0102202E308A0102200D3064
:100720008A0102200A308A010220CA01CB014A084C
:10073000A0004B08A100A30196308A01D7208A119E
:10074000031DF02B8517831685138312C430860092
:1007500005308A01A9208513831685138312051796
:10076000831605138312C430860005308A01A92040
:10077000051383160513433083128A0102204F307C
:100780008A01022055308A0102204E308A0102205F
:1007900054308A01022045308A01022052308A01F9
:1007A00002202E308A0102202E308A0102202E30B3
:1007B0008A010220A9014A08A4004B08A5000130C3
:1007C000B000B1018A011C200D308A0102200A30DC
:1007D0008A010220CA0A0319CB0A8A11031D972B2A
:1007E0008A01A32AC401C5014408A0004508A1004C
:1007F000A30132308A01D7208A11031D392C8517B5
:100800008316851383124608A0004708A100003014
:100810008A01CA20D800D9018A01FF228A01272330
:1008200008308A01A920FF308600851383168513BE
:10083000831205178316051383124608A000470884
:10084000A10001308A01CA20D800D9018A01FF2203
:100850008A01272308308A01A920FF30860005136A
:10086000831605138312C40A0319C50A8A11031DCE
:10087000F42B0800C401C5014408A0004508A100EC
:100880005108A30050088A01D7208A11031D822C29
:1008900085178316851383124608A0004708A10018
:1008A00000308A01CA20D800D9018A01FF228A01BA
:1008B000272308308A01A920FF308600851383167C
:1008C0008513831205178316051383124608A000AB
:1008D0004708A10001308A01CA20D800D9018A0145
:1008E000FF228A01272308308A01A920FF308600D1
:1008F0000513831605138312C40A0319C50A8A1146
:10090000031D3C2C08003730D800D9015808A0003E
:100910005908A100A3017F308A01D7208A11031D45
:10092000C12C85178316851306308312B6008030DC
:10093000B4005808A20004308A014A200517831623
:10094000051383128830860001308A01A92085139F
:1009500083168513831205138316051364008A1109
:100960008312851CBB2C64008A11851CB92C8A015A
:10097000B32C8A01A32AD80A0319D90A8A11031DA4
:10098000862C8A159D238A01A32A4E08A0004F08B1
:10099000A10001308A01CA20D200D3015208A00070
:1009A0005308A100A30102308A01D4208A11031D3B
:1009B000DD2C8A11512D8A11502D5208A0005308A8
:1009C000A100A30102308A01E0208A11031DEC2C52
:1009D0008A15EA2D8A11502D5208A0005308A10053
:1009E000A30103308A01E0208A11031DFB2C8A1524
:1009F000EA2D8A11502D5208A0005308A100A3012E
:100A000004308A01E0208A11031D112D3230D000FC
:100A1000D1010130A300F4308A01AA2008008A1114
:100A2000502D5208A0005308A100A30105308A01EF
:100A3000E0208A11031D272D3230D000D101013072
:100A4000A300F4308A01AA2008008A11502D520810
:100A5000A0005308A100A30106308A01E0208A11FA
:100A6000031D3D2D3230D000D1010130A300F43000
:100A70008A01AA2008008A11502D5208A0005308AC
:100A8000A100A30106308A01DA208A11031D502D2E
:100A90001930D000D1010130A300F4308A01AA201E
:100AA00008008A0183248A01512D20308A01022006
:100AB00052308A0102204F308A01022055308A01CB
:100AC00002204E308A01022044308A010220313057
:100AD0008A0102202E308A0102202E308A01022053
:100AE0002E308A0102200D308A0102200A308A014C
:100AF000022064008A11851C972D64008A11051953
:100B0000832D8A016E2B64008A118519892D8A0133
:100B10006E2B64008A11051A8F2D8A016E2B6400DA
:100B20008A110518952D8A016E2B8A01792D0F30B7
:100B3000C600C7014608A0004708A100A301003075
:100B40008A01DD208A11031D422E64008A110519D5
:100B5000AE2D0430BE00BF018A15402964008A1101
:100B60008519B72D0230BE00BF018A1540296400E7
:100B70008A11051AC02D0130BE00BF018A15402917
:100B800064008A110518C92D0330BE00BF018A1503
:100B9000402964008A11851CCF2D8A01A32A0630C2
:100BA000B6008030B4007830A2000A308A014A20B2
:100BB00043308A0102204F308A01022055308A01D9
:100BC00002204E308A01022054308A010220453032
:100BD0008A01022052308A0102202E308A0102202E
:100BE0002E308A0102202E308A010220A9014608F7
:100BF000A4004708A5000130B000B1018A011C2003
:100C00000D308A0102200A308A01022044308A0114
:100C1000022049308A01022047308A0102204930EF
:100C20008A01022054308A01022053308A010220B6
:100C30002E308A0102202E308A0102202E308A01B5
:100C40000220A9015E08A400A5010130B000B10195
:100C50008A011C20A9015F08A400A5010130B00091
:100C6000B1018A011C200D308A0102200A308A015C
:100C700002208A013A240130C602031CC7028A11ED
:100C800003189A2D8A01832C4E08A0004F08A1005A
:100C90008A0184202008CE002108CF003E08A00051
:100CA0003F08A100A30101308A01E0208A11031D41
:100CB000762E64008A110519622E0A30BE00BF012B
:100CC0008A15BF2964008A1185196B2E0730BE0072
:100CD000BF018A15BF2964008A110518742E0630D9
:100CE000BE00BF018A15BF298A11EC2E3E08A00064
:100CF0003F08A100A30102308A01E0208A11031DF0
:100D00009E2E64008A1105198A2E0530BE00BF018F
:100D10008A15BF2964008A11051A932E0730BE0078
:100D2000BF018A15BF2964008A1105189C2E09305D
:100D3000BE00BF018A15BF298A11EC2E3E08A00013
:100D40003F08A100A30103308A01E0208A11031D9E
:100D5000C62E64008A110519B22E0830BE00BF01EC
:100D60008A15BF2964008A118519BB2E0930BE007F
:100D7000BF018A15BF2964008A11051AC42E0630E6
:100D8000BE00BF018A15BF298A11EC2E3E08A000C3
:100D90003F08A100A30104308A01E0208A11031D4D
:100DA000EC2E64008A118519DA2E0530BE00BF01D1
:100DB0008A15BF2964008A11051AE32E0A30BE0085
:100DC000BF018A15BF2964008A110518EC2E08306E
:100DD000BE00BF018A15BF2943308A0102204F306F
:100DE0008A01022055308A0102204E308A010220F9
:100DF00054308A01022045308A01022052308A0193
:100E000002202E308A0102202E308A0102202E304C
:100E10008A010220A9014608A4004708A500013064
:100E2000B000B1018A011C200D308A0102200A3075
:100E30008A01022044308A01022049308A010220BE
:100E400047308A01022049308A01022054308A0149
:100E5000022053308A0102202E308A0102202E30D7
:100E60008A0102202E308A010220A9015E08A40016
:100E7000A5010130B000B1018A011C20A9015F0861
:100E8000A400A5010130B000B1018A011C200D3081
:100E90008A0102200A308A01022008008A01832C7C
:100EA0004E08A0004F08A1008A0184202008CE002F
:100EB0002108CF003E08A0003F08A100A301053093
:100EC0008A01E0208A11031D792F64008A11051A16
:100ED0006E2F0B30BE00BF018A153E2A64008A11B6
:100EE0000518772F0C30BE00BF018A153E2A8A15DF
:100EF00012283E08A0003F08A100A30106308A0185
:100F0000E0208A11031D982F64008A1105198D2F86
:100F10000D30BE00BF018A153E2A64008A11851972
:100F2000962F0E30BE00BF018A153E2A8A15122860
:100F30003E08A0003F08A100A30107308A01E0207D
:100F40008A11031DB72F64008A110519AC2F0B30CD
:100F5000BE00BF018A153E2A64008A110518B52F0C
:100F60000E30BE00BF018A153E2A8A1512283E089F
:100F7000A0003F08A100A30108308A01E0208A11E7
:100F8000031DD62F64008A118519CB2F0D30BE00AA
:100F9000BF018A153E2A64008A11051AD42F0D302C
:100FA000BE00BF018A153E2A8A1512283E08A000FD
:100FB0003F08A100A30109308A01E0208A11031D26
:100FC000F52F64008A110519EA2F0C30BE00BF010D
:100FD0008A153E2A64008A11051AF32F0E30BE00CE
:100FE000BF018A153E2A8A1512283E08A0003F0834
:100FF000A100A3010A308A01E0208A15031D1228EE
:1010000064008A15851909280B30BE00BF018A15B6
:101010003E2A64008A15051812280D30BE00BF0153
:101020008A153E2A0630B6008030B4007830A2001F
:101030000A308A014A2043308A0102204F308A0157
:10104000022055308A0102204E308A01022054309D
:101050008A01022045308A01022052308A01022092
:101060002E308A0102202E308A0102202E308A0181
:101070000220A9014608A4004708A5000130B000DD
:10108000B1018A011C200D308A0102200A308A0138
:10109000022044308A01022049308A010220473070
:1010A0008A01022049308A01022054308A0102203C
:1010B00053308A0102202E308A0102202E308A010C
:1010C00002202E308A010220A9015E08A400A50199
:1010D0000130B000B1018A011C20A9015F08A40001
:1010E000A5010130B000B1018A011C200D308A0138
:1010F00002200A308A01022008008A01832C4E084F
:10110000A0004F08A1008A0184202008CE002108F9
:10111000CF003E08A0003F08A100A3010B308A01C8
:10112000E0208A15031D9C2864008A1505189A285A
:101130008A15BD2A8A15D3283E08A0003F08A100C1
:10114000A3010C308A01E0208A15031DAF2864003A
:101150008A15051AAD288A15BD2A8A15D3283E0896
:10116000A0003F08A100A3010D308A01E0208A15EC
:10117000031DC22864008A158519C0288A15BD2A56
:101180008A15D3283E08A0003F08A100A3010E3015
:101190008A01E0208A15031DD32864008A150519E9
:1011A000D3288A15BD2A0630B6008030B4007830C6
:1011B000A2000A308A014A2043308A0102204F30BF
:1011C0008A01022055308A0102204E308A01022015
:1011D00054308A01022045308A01022052308A01AF
:1011E00002202E308A0102202E308A0102202E3069
:1011F0008A010220A9014608A4004708A500013081
:10120000B000B1018A011C200D308A0102200A3091
:101210008A01022044308A01022049308A010220DA
:1012200047308A01022049308A01022054308A0165
:10123000022053308A0102202E308A0102202E30F3
:101240008A0102202E308A010220A9015E08A40032
:10125000A5010130B000B1018A011C20A9015F087D
:10126000A400A5010130B000B1018A011C200D309D
:101270008A0102200A308A01022008008A01832C98
:101280008A01C52420308A01022043308A010220CD
:1012900041308A0102204C308A01022043308A0109
:1012A000022031308A0102202E308A0102202E30A5
:1012B0008A0102202E308A0102200D308A0102208C
:1012C0000A308A0102200630B6008030B400643053
:1012D000A20050308A014A204608C6004708C700CD
:1012E0004608A0004708A100A30100308A01DD20C4
:1012F0008A15031DBD290630B6008030B400783051
:10130000A2000A308A014A208A0144268A013A242E
:1013100043308A0102204F308A01022055308A0171
:1013200002204E308A01022054308A0102204530CA
:101330008A01022052308A0102202E308A010220C6
:101340002E308A0102202E308A010220A9014A088B
:10135000A4004B08A5000130B000B1018A011C2097
:101360000D308A0102200A308A0102200130C602B3
:10137000031CC7028A15031870298A01832C8A016D
:10138000C52420308A01022043308A0102204130E6
:101390008A0102204C308A01022043308A01022057
:1013A00032308A0102202E308A0102202E308A013A
:1013B00002202E308A0102200D308A0102200A30DC
:1013C0008A0102200630B6008030B4006430A200EA
:1013D00050308A014A204608C6004708C700460820
:1013E000A0004708A100A30100308A01DD208A1572
:1013F000031D3C2A0630B6008030B4007830A200CD
:101400000A308A014A208A013A2443308A010220A4
:101410004F308A01022055308A0102204E308A0165
:10142000022054308A01022045308A0102205230C5
:101430008A0102202E308A0102202E308A010220E9
:101440002E308A010220A9014A08A4004B08A500F9
:101450000130B000B1018A011C200D308A01022048
:101460000A308A0102208A0150270130C602031C7B
:10147000C7028A150318EF298A01832C8A01C52423
:1014800020308A01022043308A01022041308A0143
:1014900002204C308A01022043308A01022033307E
:1014A0008A0102202E308A0102202E308A01022079
:1014B0002E308A0102200D308A0102200A308A0172
:1014C00002200630B6008030B4006430A2005030F4
:1014D0008A014A204608C6004708C7004608A000FF
:1014E0004708A100A30100308A01DD208A15031DF1
:1014F000BB2A0630B6008030B4007830A2000A3033
:101500008A014A208A013A248A157F2043308A01C1
:1015100002204F308A01022055308A0102204E30CD
:101520008A01022054308A01022045308A010220BB
:1015300052308A0102202E308A0102202E308A0188
:1015400002202E308A010220A9014A08A4004B087B
:10155000A5000130B000B1018A011C200D308A01C4
:1015600002200A308A0102200130C602031CC70291
:101570008A1503186E2A8A01832C8A01C52420301B
:101580008A01022043308A01022041308A01022070
:101590004C308A01022043308A01022034308A0113
:1015A00002202E308A0102202E308A0102202E30A5
:1015B0008A0102200D308A0102200A308A010220AD
:1015C0000630B6008030B4006430A20050308A018A
:1015D0004A204608C6004708C7004608A00047083A
:1015E000A100A30100308A01DD208A15031D382BDC
:1015F0000630B6008030B4007830A2000A308A018C
:101600004A208A013A2443308A0102204F308A015D
:10161000022055308A0102204E308A0102205430C7
:101620008A01022045308A01022052308A010220BC
:101630002E308A0102202E308A0102202E308A01AB
:101640000220A9014A08A4004B08A5000130B000FF
:10165000B1018A011C200D308A0102200A308A0162
:1016600002200130C602031CC7028A150318ED2AA6
:101670008A01832C6430BA00BB010A30B800B9017A
:101680003808A0003908A100A30100308A01DD203C
:101690008A15031D9C2B0630B6008030B4005A30EA
:1016A000A20010308A014A203B08A3003A088A01B0
:1016B000AA200630B6008030B4005E30A2001030A0
:1016C0008A014A203B08A3003A088A01AA20063072
:1016D000B6008030B4006130A20010308A014A2088
:1016E0003B08A3003A088A01AA200630B6008030E1
:1016F000B4006330A20010308A014A203B08A300E6
:101700003A088A01AA2064008A15851C8F2B640080
:101710008A15851C8D2B8A15872B8A01A32A0830F0
:10172000BA020030031C013EBB020130B802031CA8
:10173000B9028A150318402B08000630B600803025
:10174000B4005A30A20028308A014A2050308A0161
:10175000A9200630B6008030B4005A30A2002830EC
:101760008A014A203C308A01A9200630B600803028
:10177000B4005830A2000A308A014A2014308A018D
:10178000A9200630B6008030B4005A30A2002830BC
:101790008A014A2050308A01A9200630B6008030E4
:1017A000B4006030A20028308A014A2014308A0137
:1017B000A9200630B6008030B4005E30A20014309C
:1017C0008A014A2014308A01A9200630B6008030F0
:1017D000B4005E30A20028308A014A2050308A01CD
:1017E000A9200630B6008030B4005A30A200143070
:1017F0008A014A2014308A01A9200630B6008030C0
:10180000B4005A30A20028308A014A2032308A01BE
:10181000A9200630B6008030B4005830A200143041
:101820008A014A2014308A01A9200630B60080308F
:10183000B4005A30A20028308A014A2008008513DB
:10184000831685138312051383160513063083123E
:10185000B6008030B4005808A20004308A014A2043
:101860000130D8020030031C013ED90285178316CF
:1018700085138312FE30860032308A01A920851339
:10188000831685138312FF30860032308A01A92027
:101890000630B6008030B4005808A20004308A0137
:1018A0004A200130D8020030031C013ED90205173E
:1018B000831605138312BF30860032308A01A920B7
:1018C000051383160513323083128A01A9200630CE
:1018D000B6008030B4005808A20004308A014A20C3
:1018E0000130D8020030031C013ED902851783164F
:1018F00085138312F730860032308A01A9208513C0
:10190000831685138312FF30860032308A01A920A6
:101910000630B6008030B4005808A20004308A01B6
:101920004A200130D8020030031C013ED9020517BD
:10193000831605138312EF30860032308A01A92006
:10194000051383160513323083128A01A92006304D
:10195000B6008030B4005808A20004308A014A2042
:101960000130D8020030031C013ED90285178316CE
:10197000851383128030860032308A01A9208513B6
:10198000831685138312FF30860032308A01A92026
:101990000630B6008030B4005808A20004308A0136
:1019A0004A200130D8020030031C013ED90205173D
:1019B000831605138312FB30860032308A01A9207A
:1019C000051383160513323083128A01A9200630CD
:1019D000B6008030B4005808A20004308A014A20C2
:1019E0000130D8020030031C013ED902851783164E
:1019F00085138312DF30860032308A01A9208513D7
:101A0000831685138312FF30860032308A01A920A5
:101A10000630B6008030B4005808A20004308A01B5
:101A20004A200130D8020030031C013ED9020517BC
:101A3000831605138312FE30860032308A01A920F6
:101A4000051383160513323083128A01A92006304C
:101A5000B6008030B4005808A20004308A014A2041
:101A60000130D8020030031C013ED90285178316CD
:101A700085138312EF30860032308A01A920851346
:101A8000831685138312FF30860032308A01A92025
:101A90000630B6008030B4005808A20004308A0135
:101AA0004A200130D8020030031C013ED90205173C
:101AB0008316051383127F30860032308A01A920F5
:101AC000051383160513323083128A01A9200630CC
:101AD000B6008030B4005808A20004308A014A20C1
:101AE0000130D8020030031C013ED902851783164D
:101AF00085138312FD30860032308A01A9208513B8
:101B0000831685138312FF30860032308A01A920A4
:101B10000630B6008030B4005808A20004308A01B4
:101B20004A200130D8020030031C013ED9020517BB
:101B3000831605138312EF30860032308A01A92004
:101B4000051383160513323083128A01A92006304B
:101B5000B6008030B4005808A20004308A014A2040
:101B60000130D8020030031C013ED90285178316CC
:101B700085138312FD30860032308A01A920851337
:101B8000831685138312FF30860032308A01A92024
:101B90000630B6008030B4005808A20004308A0134
:101BA0004A200130D8020030031C013ED90205173B
:101BB000831605138312DF30860032308A01A92094
:101BC000051383160513323083128A01A920FF30D2
:101BD00086000800B801B9013808A0003908A10042
:101BE000A30164308A01D7208A15031D312E851781
:101BF0008316851383124608A0004708A100003011
:101C00008A01CA20D800D9018A01FF228A0127232C
:101C100008308A01A920FF308600851383168513BA
:101C2000831205178316051383124608A000470880
:101C3000A10001308A01CA20D800D9018A01FF22FF
:101C40008A01272308308A01A920FF308600051366
:101C5000831605138312B80A0319B90A8A15031DDE
:101C6000EC2D8A153A238A151F248A15EA2D423055
:101C70008A0102204F308A0102204D308A01022061
:101C800042308A01022020308A01022047308A0136
:101C9000022041308A0102204D308A010220453065
:101CA0008A01022020308A01022056308A01022057
:101CB00031308A0102202E308A01022030308A0120
:101CC00002200D308A0102200A308A0102200D30E4
:101CD0008A0102200A308A0102204D308A01022046
:101CE00041308A01022044308A01022045308A01B5
:101CF000022020308A01022042308A01022059301D
:101D00008A01022020308A01022052308A010220FA
:101D100055308A01022049308A01022020308A0190
:101D2000022043308A01022041308A0102204230E1
:101D30008A01022052308A01022041308A010220A9
:101D40004C308A01022020308A01022032308A0180
:101D5000022030308A01022031308A0102203030E6
:0A1D60008A01022063008A15B22EEA
:02400E00383F39
:00000001FF
